:100000008A110A1205280000090083169F01831235
:10001000073099008B1383160510851005110516FE
:100020008312B101B201AE016330AF000130B00004
:100030000510851405112E08013C031D2C280514FC
:10004000851405152F08A000A10199208510051120
:100050003008A000A10199201F30830505102E084B
:10006000003C031D4E283108013EB1003208031840
:10007000013E003EB2003108A0003208A10013305A
:10008000A30088307720031D4C2883168510831227
:1000900002308506B101B2011F3083051F30830590
:1000A00053201B285228051A73282C30A000013039
:1000B000A10099202E08003C031D62280130AE00EB
:1000C0008130AF001F3083052F08093C031D6B28CA
:1000D000AE018130AF001F3083051E302F02AF000C
:1000E0002F08643CB0001F30830508007628A2006A
:1000F00005308928A20002308928A200063089280C
:10010000A20003308928A20004308928A20001300F
:100110008928A80023082102031D90282208200214
:10012000043003180130031902302805031DFF3085
:100130000800A0080319A428AB20A00300000000B9
:100140000000000000009928A10803190800AB2056
:10015000A103A00399280C30A500A50BAD28000031
:1001600000001230A200A20BBA28BC20BC20000064
:1001700000000800BC20B3280D30A400A40BBE284A
:040180000000080073
:02400E00C433B9
:00000001FF
